:100000000EC026C037C024C023C022C021C020C0DB
:100010001FC01EC01DC01CC01BC01AC019C01124A7
:100020001FBECFEDCDBF10E0A0E6B0E0ECE7F3E0FF
:1000300002C005900D92A236B107D9F720E0A2E6E2
:10004000B0E001C01D92AC3AB207E1F714D094C100
:10005000D7CF23E030E091E0482F50E0092E02C0D6
:10006000559547950A94E2F78427990F2150310955
:1000700099F7089508958FE188BB80E28BBFE0E097
:10008000F0E089E080935700E491E7FD0FC0809194
:1000900060009091610097FD0796A3E09595879584
:1000A000AA95E1F79093610080936000EF70E430CF
:1000B00079F4809160009091610097FDCF96F6E011
:1000C00095958795FA95E1F790936100809360008C
:1000D00080E090E046D1809367008230F1F781E0C4
:1000E00090E047D1182F809363009093640083E0E1
:1000F00090E03FD1909366008093650017FF02C0A7
:100100008DE101C089E18093620013FF02C0C398B2
:10011000BB9A209163003091640020763327E4E09D
:1001200036952795EA95E1F781E090E002C0880FC7
:10013000991F2A95E2F74091600050916100019764
:1001400068F430E1C32E00ED17E040E2D42E5FE109
:10015000B52E67E1A62E78E0972E48C02BE02150FF
:1001600071F3FA013197F1F7FACFB39BFECF86B363
:1001700082958170C82F80E0D82FE0FC3EC08C2F84
:10018000E4FC67DFEE249FE0F9228F0D8F70F82EDC
:1001900085E090E0E6D0F816A0F1C5BAB09BC3C0E8
:1001A000809162008DB90000809162008DB90000DD
:1001B0008091630083FFC3C0A8BA97BADBBE85B73E
:1001C000877E806185BFF89485B7806285BF78940B
:1001D000889585B78F7D85BF8091630081FD06C0BE
:1001E00080916000909161000197F1F7E0906300C9
:1001F000F0906400E3FCBBCFB8CFCE0121E08227B2
:10020000BFCF8F2D90E00396880F991FB2D07C014D
:1002100001969093AB008093AA00A3D08093A9008D
:10022000482F50E0B7016E5F7F4F89E690E08AD09B
:100230008091630087FF02C0C29801C0C29ABA9A37
:1002400090E08091A900981708F0A7CFE92FF0E07F
:10025000E759FF4F80818093680080E0209168001B
:10026000821708F054C01EB8DF01A80FB11D119607
:100270002C912FB9209162002DB981110AC02091D3
:10028000630023FF02C0C39A01C0C39827B32E6046
:1002900027BB209162002DB90000209162002DB98A
:1002A0000000209162002DB90000209162002DB95C
:1002B0000000209162002DB90000209162002DB94C
:1002C0000000209162002DB90000209162002DB93C
:1002D0000000209162002DB90000209162002DB92C
:1002E0000000209162002DB90000209162002DB91C
:1002F0000000209162002DB90000209162002DB90C
:100300000000209162002DB900008F5FA7CF80917F
:10031000630083FF02C0C39801C0C39A8091680044
:100320008F5F980F8ECF809163009091640097FF4C
:1003300037CFC8010197F1F7A89ADABE31CFB8BA22
:1003400017BA3CCFA82F862FE82FE199FECF1FBA0E
:1003500005C0EEBBE09AE3950DB20D924150C8F78F
:100360000895E199FECF1FBA8EBBE09A99278DB30D
:0C0370000895A8E142E0E8CFF894FFCF28
:02037C00204E11
:00000001FF
